:020000040000FA
:0600000079EF1CF0120074
:0600080004EF08F01200F5
:060018000CEF08F01200DD
:0610000079EF1CF0120064
:0610080004EF1BF01200D2
:0610180006EF1BF01200C0
:06102A0003004439000040
:10103000A20000000500000041390000FD02000090
:10104000030000003839000099000000090000008A
:10105000400EE66E000EE66E020EE66EB0EC17F085
:10106000E552E552E55200090DE060C085F000014F
:101070009B5103E085C0E6FF09D085C0E6FFA7ECE1
:101080000CF005D000019B5104E0E66AC4DBE55298
:1010900012009B5112E18B50800B0FE19FC00BF0AF
:1010A000A0C00CF09F07000EA05B0B500C1005E1D8
:1010B000E66887EC1CF0E552C0D812008BBE04D065
:1010C00000019F69A0695CD092929290929892964A
:1010D0009294929A89808982936800000000898A9C
:1010E000000000000A0EE66E87EC1CF0E5520000DE
:1010F000000089980000000089868984FE0EE66E53
:1011000087EC1CF0E552FE0EE66E87EC1CF0E55213
:101110008B9E320EE66E62EC1CF0E55200019F6978
:10112000A0690001010E996F89968998936A010E52
:10113000E66E87EC1CF0E55281680000000089949F
:10114000010EE66E87EC1CF0E55289840000000079
:10115000010EE66E87EC1CF0E552FE0E816E00007B
:1011600000008994010EE66E87EC1CF0E55289843C
:1011700000000000936889888986899889908992FF
:10118000120092929290929892969294929A89805A
:101190008982936800000000898A000000000A0E1E
:1011A000E66E87EC1CF0E552000000008998000014
:1011B000000089868984FE0EE66E87EC1CF0E552FD
:1011C000FE0EE66E87EC1CF0E5528B9E00019951F5
:1011D00005E1320EE66E62EC1CF0E55200019F69FB
:1011E000A0690001010E996F89968998936A010E92
:1011F000E66E87EC1CF0E5528168000000008994DF
:10120000010EE66E87EC1CF0E552898400000000B8
:10121000010EE66E87EC1CF0E55200000000899498
:10122000010EE66E87EC1CF0E55289840000000098
:101230009368898889868998120089968998936A23
:10124000010EE66E87EC1CF0E5528168000000009C
:101250008994010EE66E87EC1CF0E552898400004B
:101260000000010EE66E87EC1CF0E552FE0E816E6A
:10127000000000008994010EE66E87EC1CF0E55238
:1012800089840000000093688998898689988990EC
:101290000001996BF18E8992899089988996899439
:1012A000899A9282928092889286928493680A0E9A
:1012B000E66E87EC1CF0E5528B8E1200AEDBE65238
:1012C000FE0EDB50DF6EDF98DF9ADF9CDF9EFE0EA6
:1012D000DB90DB92DB94DB96DB380F0BE76EFE0EC8
:1012E000E7CFDBFFDB50EEDBF5CF7FF0DF50EADB53
:1012F000F5CF80F0E55296D39368898A89848986F0
:101300008998899A898A000000008994010EE66E06
:1013100087EC1CF0E55289840000000089988986DA
:101320000A0EE66E87EC1CF0E552936A8A6A0A0E92
:10133000E66E87EC1CF0E552000000008994010E77
:10134000E66E87EC1CF0E552898400000000200E58
:101350008A6E0A0EE66E87EC1CF0E5520000000073
:101360008994010EE66E87EC1CF0E552898400003A
:1013700000000A0EE66E87EC1CF0E552936889883F
:101380000A0EE66E87EC1CF0E552815000D0120088
:10139000000000008994010EE66E87EC1CF0E55217
:1013A000898400000000815000D01200D9CFE6FFF0
:1013B000E1CFD9FF899A898489868998010EE66EE2
:1013C00087EC1CF0E552898A0A0EE66E87EC1CF069
:1013D000E552936A816A020EE66E87EC1CF0E552D4
:1013E000000000008994010EE66E87EC1CF0E552C7
:1013F000898400000000020EE66E87EC1CF0E552C6
:10140000000000008994010EE66E87EC1CF0E552A6
:10141000898400000000FE0EDB50816E020EE66E35
:1014200087EC1CF0E552000000008994010EE66E86
:1014300087EC1CF0E552898400000000020EE66E85
:1014400087EC1CF0E5529368F19E8988010EE66EE8
:1014500087EC1CF0E552E552E7CFD9FF1200D9CF57
:10146000E6FFE1CFD9FF8984898689980A0EE66E66
:1014700087EC1CF0E552936A8A6A000000008994A8
:10148000010EE66E87EC1CF0E55289840000000036
:10149000000000008994010EE66E87EC1CF0E55216
:1014A000898400000000FE0EDB508A6E0000000000
:1014B0008994010EE66E87EC1CF0E55289840000E9
:1014C000000093688988E552E7CFD9FF1200D9CF91
:1014D000E6FFE1CFD9FFE6528150DF6E0000000049
:1014E0008994010EE66E87EC1CF0E55289840000B9
:1014F0000000DF5000D0E552E552E7CFD9FF1200DF
:10150000560E0201005D10E1560E015D0DE1000175
:1015100061510FE10001E40E626F340E636F000150
:10152000030E11DB010E04D00001615102E171DAFA
:10153000616F00019B6B120070DA00019B5105E1A5
:1015400000C27AF0010E9B6F08D000C27BF09B6B4B
:101550007AC000F27BC001F2D3DF64D25EDAA4DA93
:101560002BE10001795191DA01E694DA17E3DF6AA1
:10157000DF508BDA01E68EDA02E2EADAF9D700010F
:101580009C5104E00001792B00019C6B000161512A
:1015900001E156DA000179510FE10BD079517F0852
:1015A0000BE3DF6A010EDB50DF5C02E2D1DAFAD72F
:1015B0004FDA0001100E9B6F020EE15C02E2E16A5D
:1015C000E552E16E2FD229DA6FDA2BE10001795171
:1015D0005CDA01E65FDA17E3DF6ADF5056DA01E62C
:1015E00059DA02E2BBDAF9D700019C5104E00001AC
:1015F000792B00019C6B0001615101E121DA0001AE
:1016000079510FE10BD079517F080BE3DF6A010EAE
:10161000DB50DF5C02E2A2DAFAD71ADA0001100E20
:101620009B6F020EE15C02E2E16AE552E16EFAD1E3
:1016300076DA520E0201012502250325E76E020E1D
:10164000E7CFDBFFDB50045D08E00001615102E100
:10165000E0D9616F00019B6B1FD002C2DFFF010E5A
:1016600003C2DBFF01C279F00001795104E179691D
:101670000001010E9C6FDF501F0806E300019D6B07
:10168000030E9B6FA0DF08D0010EDBCFE6FFDFCF9C
:10169000E6FFE5DE1EDA62DF030EE15C02E2E16AEC
:1016A000E552E16EBFD13BDA450E0201012502256C
:1016B00003250425E76E020EE7CFDBFFDB50055D57
:1016C00008E00001615102E1A4D9616F00019B6B48
:1016D00026D003C2DFFF010E04C2DBFF01C279F096
:1016E0000001795104E179690001010E9C6F02014A
:1016F000025102E1899003D0020503E189808992B9
:1017000007D0020E025D02E1899001D089808982B2
:10171000010EDBCFE6FFDFCFE6FF48DEDAD9030EAE
:10172000E15C02E2E16AE552E16E7CD1EAD9FE0EAB
:10173000DB50DF5C16E2010EDBCFF3FFDB2AF35058
:10174000EA6A000FE96E020EEA22EF50E66E00012F
:101750009A519A2BEA6A7A0FE96E000EA0D9DF2A15
:10176000E6D7020EE15C02E2E16AE552E16E5AD18F
:10177000C8D9FE0EDB50DF5C14E2010EDB50EA6AD2
:101780007A0FE96E000EEA22EF50E66E010EDB5092
:10179000EA6A000FE96E020E82D9010EDB2ADF2A07
:1017A000E8D700019A6B020EE15C02E2E16AE552C1
:1017B000E16E38D10001615104E102014F0E406F2A
:1017C00035D9120002010151520A0DE0170A04E056
:1017D000000161511DE11BD0450E025D1BE10001BE
:1017E000615118E106D0520E025D0AE1000161511B
:1017F0000DE10201080E406F416F97D9020E88D1AA
:1018000002C2E6FFE9EC19F0E552D4DF1200FBD882
:1018100000019B6B120001D9E65200019B51100A96
:1018200001E188D0190A74E0010A4DE00F0A30E0A6
:10183000010A28E0020A21E0070A1AE0010A0CE086
:10184000030A05E00001615101E07DD07BD0FE0E6E
:10185000DBCFE6FF71DE5AD0050E9A5D02E32CD98C
:1018600001D03ED9050E00019A5D6FE325D96DD0F8
:10187000000161516AE1A7DE68D00001615165E1B4
:101880006DDE63D0FE0EDBCFE6FF87EC13F03ED0BB
:10189000FE0EDB5006E1F0D858E10001615153E142
:1018A0001AD0510E0201005D0AE10001080E9B6F83
:1018B000000161514AE1A50EE66E350E26D0000109
:1018C000615143E11FD0FE0EDB500BE1D5D83DE165
:1018D0000001615138E1D30EE66E350E07D9E552AD
:1018E00032D05A0E0201005D0AE10001090E9B6F21
:1018F000000161512AE1EA0EE66E340E06D00001C5
:10190000615123E1D30EE66E350EF0D8E5521DD0BD
:10191000A96AAA0EA86EA69EA69CA684550EA76EBE
:10192000AA0EA76EA682050EE66E87EC1CF0E552A5
:10193000A69409D00001615108E19EC040F276D81A
:101940009E6B03D060D800019B6BE5526BD065D8CD
:10195000E652DF6A02010051450A3CE0040A2FE02A
:10196000310A45E0200A43E0030A41E0240A3FE04F
:101970002F0A3DE00F0A1AE0250A39E0300A14E088
:10198000100A0BE0040A04E00001615130E12ED09E
:10199000020E6BD82CE3B4DD2AD05EEC08F0040E06
:1019A00064D81FE345DE23D00DDF21D05EEC08F0C4
:1019B000FE0EDBCFE6FF1BEC13F0E55218D0000162
:1019C000615105E1770EE66E350E90D8E5520001C3
:1019D000070E0AD0C1EC08F0040E47D802E363DE1C
:1019E00006D07ED80001020E9B6F01D00CD8E552C4
:1019F00019D081D8EA22EF5000019E259E6F000188
:101A00007907DF2A120098D8020E9DD8010E616F67
:101A1000120092D8010EA3EF0DF0D9CFE6FFE1CF6F
:101A2000D9FF1200E552E7CFD9FF12007ED8010E90
:101A3000666F0001676F0001616F00019B6B120010
:101A40000001000E626F010E636F0001800E60D016
:101A50000001000E626F010E636F010EDBCF66F0B6
:101A60000001676F0001616F1200F36EFE0EDBCFA5
:101A7000F4FFF350F45C1200A12B640EE66E62ECEE
:101A80001CF0E5520001A15112000B6E0C6AD890B7
:101A90000C501200800E0B5C000E0C581200EA2253
:101AA000E552E750EF6E1200020EE126010E79C0FA
:101AB000DBFF000161511200050EE66E59DEE552B2
:101AC00018EF0BF0F76AD30FF66E340EF72208000A
:101AD0001200E552E55200019D6B040E9B6F12004F
:101AE000FE0EDBCFE6FF22DEE5521200E66E1BECB7
:101AF00018F0E5521200DF50EA6A000FE96E010E9D
:101B000012008BDF020EE126010EDB6ADF6A120093
:101B1000666F0001010E676F0001616F12007DDFCB
:101B2000030EE126020EDB6A12000001400E626F16
:101B3000020E636F000112000001E70E626F340EA7
:101B4000636F00011200666F0001676B00011200F5
:101B5000BEDCE66ED0DFA3DFF9EF0CF0CCDFEA22CB
:061B6000EF68F9EF0CF044
:0A1B660084EC12F06A6A686A9F0EB0
:101B70006B6EFB0E696E6D8C6D9C6E6A5FEC12F085
:101B8000DF6ADF500B6E0C6A100E0B5C000E0C58F7
:101B900010E2DF50040DF3CFE9FFF4CFEAFF000EAF
:101BA000E926040EEA22EE6AEE6AEE6AEE6ADF2A9F
:101BB000E8D7160E706E68A604D0030E29EC12F05A
:101BC000FAD70201DE6BE36BE46BE56B6D98080EF0
:101BD000D26F040ED36FC46BC36B87EF12F084EC2B
:101BE00012F00201C3510BE16D6A696A6DB602D051
:101BF0006D86FCD70201010EC36F160E6F6EC30512
:101C000008E16DBA06D0686A696A69806988020E5F
:101C1000C36F6850040B04E06950040B01E065D801
:101C20006DB249D06850010B11E06950010B0EE014
:101C30009ADF0201040EC36F0401400E026F040E0E
:101C4000036F080E016F006B8C0E00136850100BB1
:101C500004E06950100B01E042D86850400B08E0E6
:101C60006950400B05E076EC1BF0060E29EC12F0F3
:101C70006850200B04E06950200B01E01ED868502A
:101C8000020B06E06950020B03E077EC1BF06A6A76
:101C9000040E0201C35D0FE369A60DD0DF6A040ED6
:101CA000DF5C09E268A607D06CCFEBF2030ED1DB54
:101CB00026D8DF2AF4D787EF12F070A00DD050ECB1
:101CC00012F0EF50800807E1CEDBEF50840803E10B
:101CD000E7DB8C0EEF6E7090050E29EF12F0698431
:101CE000040EB7DB6D8274EF1BF06D9275EC1BF088
:101CF000699468A403D0020EACDBFBD71200FD0E82
:101D00000201EB1519E17E0EEB15E8407F0B040D87
:101D1000F3CFC6F2F4CFC7F2000EC627040EC723D6
:101D2000C6C2C8F2C7C2C9F2C875F0EC12F002E12F
:101D3000A2EF0EF0B3EF0EF0FD0EEB15040801E17B
:101D40001AD8120090DBEF50800B02E08CDBEF6AB8
:101D50000201DA6BDB6BDF6BE06BDE6B96D878EC45
:101D60001BF071EF10F0020E0201DB5D02E1FBEFF0
:101D700010F0E7EF0EF0C8DB76DBEF50400B01E030
:101D8000010EDF6E0201D275080EC35D09E142C487
:101D90006EFF6E50000802E2100E01D0040EC36FF9
:101DA000DB0513E1E2EC12F0D4D9020E0201DA5D98
:101DB00003E159DB840E07D0DF5003E154DBC80E8A
:101DC00002D051DB880EEF6E01D001D8A0D3DDEC3C
:101DD00012F0030EE126020E0201DB5D2CE16D50D4
:101DE000100B29E05DDBEE52EF500B6E0C6A080E13
:101DF0000B1821E10C501FE1F0EC12F01CE1BEDBEE
:101E0000EF50800B18E1BADBCCDBDF6ADF500B6EE2
:101E10000C6A080E0B5C000E0C5822E2DF507FDBD0
:101E2000DF50EA6A400FE96E040EEA22E552E750FD
:101E3000EF6EDF2AEBD7DB6BBADBEF6A040ED21949
:101E40000B6ED3C20CF0010E0BC0DBFF020ED3C22F
:101E5000DBFF010EDBCFE9FF020EDBCFEAFFEF6A0B
:101E60000201E3AF0CD0E651E71107E005D0E7C26D
:101E7000FAFF0201E651F96EFADF0201E39F030E59
:101E8000E15C02E2E16AE552FCD204014051600BE0
:101E9000E842E842E842E842E842000901E0120074
:101EA00041510C0A43E00B0A3FE00C0A31E0010A01
:101EB00022E00B0A1EE0020A1CE0030A18E0080AEE
:101EC00010E0010A0CE00F0A08E0030A01E012002A
:101ED0000201DE8F080EC36F1200FDEF0FF054EF0A
:101EE00011F00201C40EDC6F020EDD6F0CD038EF72
:101EF00010F097EF0FF044510201DC6FDD6BC50E5F
:101F0000DC27020EDD23DE81010EDF6FDE8F120083
:101F10000201DE8F04014451EA6AC50FE96E020E28
:101F2000EA2242C4EFFF12007AEF1BF0120045DBF9
:101F3000050EE1260401420510E140511F0B000986
:101F40000CE10201DE8F030E0401415D04E1020198
:101F5000010EEA6F02D00201EA6B0401425147E12F
:101F600040511F0B020843E144510F0B00093FE0B1
:101F70000201DE8F040EDB6A020EF36E040EDBCF6D
:101F8000F4FFF350F45C33E2F4DA040EDBCFE6FF47
:101F900004014451800B01E0010EC9DAE552E72447
:101FA000A5DA030E415D03E163DA840E1CD04451CF
:101FB0000F0B0C6A700F0B6E0F0E0C22020E0BC073
:101FC000DBFF030E0CC0DBFF020EDBCFE9FF030ECD
:101FD000DBCFEAFFEE90ED5244AF03D049DA400E7A
:101FE00002D046DAC80EEF6E040EDB2AC5D7050E06
:101FF000E15C02E2E16AE55244D2800E0401405DF8
:1020000036E10201C00EDE6F04014351030A1EE0F7
:10201000010A09E0030A29E10201240EDC6F370EF0
:10202000DD6F120E1FD09ADAE90EF626370E87DA28
:10203000020E0201F76ADC25F66EDD51F722090077
:10204000F5CFDFF20A00F5CFE0F2120087DAEB0EEF
:10205000F626370E74DADCC2F6FFDDC2F7FF0800A1
:10206000F5500201DF6FE06B12000201DE6B12001F
:1020700004DA0401486B496B40511F0B020A11E05E
:10208000030A0CE0010A1DE10201DE8F0401488110
:102090000201EA0516E10401488313D00201DE8F34
:1020A00010D00201DE8F65DA04014451800B01E09B
:1020B000010E3DDA1BDADCD9EF50040B02E0010E11
:1020C000486F0201DEAF07D0480EDC6F040EDD6FF3
:1020D000DE81020EDF6F020EE15C02E2E16AE55290
:1020E000D0D16D980201DEBF07D0E3AF02D093DA02
:1020F00028D05DDA840E26D0E3BF2AD0040140AF99
:1021000023D00201DF510401465D0201E0510401C8
:10211000475904E246C4DFF247C4E0F21AD802018C
:10212000010EDB6F8FD9B6D9800EEF6EB9D9EE52A2
:10213000080EEF6EB5D935DAB3D9800EEF6E42DAFC
:1021400092D9C80EEF6E1200020165DAC80EEF6E6A
:10215000120093D90201080EDF5D000EE0590DE276
:10216000DFC2DEFFE0C2DDFFDA5102E1010E03D083
:10217000DA0506E1020EDA6F03D0080EDE6EDD6AC4
:1021800072D9EF9270D9EF906ED9010EDB50EF1239
:102190006AD9EE52DFCFEFFF000EDB50DF5F010E9A
:1021A000DB50E05B480EE86F040EE96FDEB10FD044
:1021B000DCD91BE0DCC2F6FFDDC2F7FFDC2B000E32
:1021C000DD230800F55084D9F3E2DB06F1D7CDD941
:1021D0000CE0DCC2E9FFDDC2EAFFDC2B000EDD23F0
:1021E000EF5076D9F4E2DB06F2D7020EE15C02E2B0
:1021F000E16AE55246D141D953D9EE52EFCFDFFF24
:10220000DFCF0BF00B500201E45D000EE55903E255
:10221000E4C2DFFF09D0DF500B6E0C6AE850E45DCA
:10222000E46F0C50E559E56F010EDB6ADF50F36E89
:10223000010EDBCFF4FFF350F45C10E2010EDB5033
:102240006ED9E1C2E9FFE2C2EAFFE12B000EE22310
:10225000E552E750EF6E010EDB2AE8D7000ED8807A
:10226000E455000EE5550CE2CAD91AD9EF50400BDF
:1022700003E184D9C80E02D081D9880EEF6E0ED04A
:102280007DD98FD9E651E71107E005D0E7C2FAFF03
:102290000201E651F96EFADF0201E39F020EE15CF2
:1022A00002E2E16AE552EDD00201DE8F08D9010EAB
:1022B000E66EE66AE66AC50EE66E020E98D942C47C
:1022C000C4F20401425104E10201100EC36F120076
:1022D0000201200EC36F7BEF1BF0CFD84AD9E5D89F
:1022E000040DF3500B6E0C6A020E0F0B05E0D89034
:1022F0000C320B32E806FBE1D8900B360C36D89046
:102300000B360C367FD90B50EE260C50ED22B0D890
:10231000EF9EFD0EDB5002E159D901D05CD9EA22D3
:10232000DECFEEFFDDCFEDFFA3D8EF9CA1D8040EEA
:10233000E926000EEA22EF8C020EE15C02E2E16A7D
:10234000E5529FD09AD8FE0EDB500C6A700F0B6ED0
:102350000F0EDFD8FD0EDB50E66E8AD8E552E7504F
:10236000EE6EED6AFD0EDBA402D0E66AF0D8FD0E3B
:10237000DBA203D0010EE66EEAD8020EE15C02E2B7
:10238000E16AE5527ED079D8FE0EDB5004E10FD928
:10239000840EEF6E05D089D8F6D887D8010FF3D810
:1023A000020EE15C02E2E16AE5526BD066D8FD0EF6
:1023B000DB5002E010D901D009D9EA22EECFDEFFCE
:1023C000EDCFDDFF55D832D9FB0EDBCFEEFFFC0E93
:1023D000DBCFEDFF4DD8EE52FA0EDBCFEFFF400E14
:1023E00047D8E850EF16880E43D8E850EF12FD0E9C
:1023F000DB5002E0F0D801D0E9D8EA22EF74DECF5A
:102400000BF0DDCF0CF00BC0F3FF0CC0F4FF020E9D
:10241000E15C02E2E16AE55234D0CFD8010EF36EFE
:10242000FC0EDB5004E0D890F336E806FCE1F31C28
:102430000B6EFD0EDBCFE9FFFE0EDBCFEAFF0B508C
:10244000EF16E5D09BD8EE52080EEF6E97D816EF38
:1024500013F0E66E680EE66E0F0EE66EDEDFE552F6
:10246000E552E5521200D2C2E9FFD3C2EAFF1200E0
:10247000DECFE9FFDDCFEAFF12009FD8020EE12692
:102480001200E16EC4D0FE0EEA6ADB34FE0BEA36BF
:10249000E96E1200400EEE6E040EED6EBEEF12F00D
:1024A000C6C2E9FFC7C2EAFF1200FD0EDB50E824F6
:1024B0000D6EFE0EDB50040DF3500D241200020EC3
:1024C000E66EE66AE66A710EE66E0F0EF7EF12F040
:1024D000E66EE8C2E9FFE9C2EAFFE82B000EE92355
:1024E000E552E750EF6EDF06010E1200040DF4CF47
:1024F0000CF088D8F350EE260C50ED221200480E56
:10250000EE6E040EED6E120058D8E6521200E5523F
:102510007ED00C220BC0DEFF0CC0DDFF1200EA6A89
:10252000480FE96E040EEA22EF50E66E1200E8242E
:102530000D6E44510F0B040DF3500D241200F722C1
:102540000900F5CFDCF20A00F5CFDDF21200FE0E35
:10255000DBCFE6FFC2DEE552E55212004251F66ED5
:10256000F76AD890F636F73612004CD8EE50ED10D8
:102570001200000EDE6E040EDD6E1200C8C2E9FF0E
:10258000C9C2EAFF1200040DF3CF0BF0F4CF0CF038
:10259000000E0B26040EBDDF840E6ADFE850EF123A
:1025A000120044D8400EEE6E040EED6E12004ADFAB
:1025B00071DF8C0EEF6E33EF12F0D9CFE6FFE1CF73
:1025C000D9FF120050DF32D87FEF12F05CDFCA0E65
:1025D000E926020E120057DFD20EE926020E120083
:1025E0005FDFEF503C0BE842E8420D081200E66E58
:1025F00048EC1CF00B6E050EE15E0B50120022DF62
:102600007FEF12F0D9CFE9FFDACFEAFF1200E552EF
:10261000E7CFD9FF1200020EDB6F25DFEE52EF6A23
:1026200022DFC80EEF6EEBDFBEEF12F0020EE926DE
:06263000000EEA22120078
:0A263600CDDB030EE12600019E6BD0
:1026400000019C6B040EF36EFE0EDBCFF4FFF35023
:10265000F45C56E30001060E9B6F01C279F002C2E2
:1026600091F003C292F00001795104E1796900010F
:10267000010E9C6F570E0201012502250325000162
:102680009E6F0001915101E1F2DA200E0001915D8F
:102690000DE290510BE0C80EE66E62EC1CF0E552C4
:1026A00040DBDBD8FF0802E10001906B200E000147
:1026B000915D01E1BCDA040EDF6EFE0EDB50DF5CE3
:1026C00015E2DF508FDB010EEFCFDBFF200E0001A4
:1026D000915D06E3010EDBCFE6FF7ED8E55202D026
:1026E000010EDB50E76E020E63DBE7D700019C5161
:1026F00005E0020E00017925796F02D00001792BE7
:10270000030EE15C02E2E16AE552E16E67D361DB50
:10271000060EE126030EDB6AFE0EDB500001795D3A
:102720000CE1FE0EDB06DB505DDB020EEFCFDBFFC4
:10273000010EF36E030EF3CFDBFFDF6AFE0EDB50FC
:10274000DF5C15E2DF504EDB040EEFCFDBFF200E27
:102750000001915D06E3040EDBCFE6FF3DD8E552B4
:1027600002D0040EDB50E76E050E22DBE7D7030E26
:10277000DB5019E0020EDB5000019E5D14E142DBEC
:1027800002E10001A46B000161511FE10001320E62
:10279000626F390E636F0001010E666F0001676B97
:1027A0000001616F12D0030EDB500FE0020EDB5010
:1027B00000019E5D0AE09EC040F20001615101E10E
:1027C000EFDA20DB02E10001A46B060EE15C02E21D
:1027D000E16AE552E16E02D3D9CFE6FFE1CFD9FF3E
:1027E000FE0EDB50FF081CE10001A45119E08986B0
:1027F00000000000898800000000000000008994AB
:10280000010EE66E87EC1CF0E552898400000000A2
:1028100000000000899800000000FE0EDB5019D077
:10282000FE0EDBCFE6FF92C0E6FF91C0E6FFD1D8F7
:10283000E552E552E5520001010EA46F010EE66E6D
:1028400087EC1CF0E552FE0EDBCFE6FF9BD8E5528D
:1028500000D0E552E7CFD9FF1200D9CFE6FFE1CF94
:10286000D9FFE6529368000000008988000000004C
:102870000000000000008150DF6E00000000899819
:1028800000000000DF5000D0E552E552E7CFD9FF4D
:102890001200D9CFE6FFE1CFD9FFFE0EDB50800B4F
:1028A000E76EFE0EE7CFDBFF000000008988000026
:1028B00000008150800B0CE0FE0EDB50800808E128
:1028C00000000000899800000000010E15D00DD016
:1028D0008150800B0AE1FE0EDB5007E10000000092
:1028E000899800000000010E07D0000000008998C0
:1028F00000000000000E00D0E552E7CFD9FF120023
:1029000093680000000089880000000081AA07D0B9
:1029100000000000899800000000010E07D00000B0
:102920000000899800000000000E00D01200D9CFEE
:10293000E6FFE1CFD9FFE6520000000089880000E1
:102940000000A00E8114DF6EFE0EDB50A00BE76EC0
:10295000FE0EE7CFDBFFFE0EDB50DF5C07E1000081
:102960000000899800000000010E07D00000000060
:10297000899800000000000E00D0E552E552E7CF34
:10298000D9FF120026DAE65293680001A36BDF6AD2
:10299000080EDF5C19E23EDA13E143DA11E1B0DF41
:1029A000000910E037DA0EE13CDA0AE10001010E1D
:1029B000A36F81CF40F2FE0EDBCF41F2F00E57DA6B
:1029C0004CDF05D0DF2AE4D70001020EA36FE552E9
:1029D00005D2D9CFE6FFE1CFD9FF0001A4514DE1E7
:1029E000AA0EE66E550EE66E550EE66E85D8E552D9
:1029F000E552E552550EE66EAA0EE66E2A0EE66E1A
:102A00007BD8E552E552E552A00EE66E550EE66E15
:102A1000550EE66E71D8E552E552E55289988986E1
:102A20008984936AFD0EDB508A6E00000000899451
:102A3000010EE66E87EC1CF0E55289840000000070
:102A4000FE0EDB508A6E000000008994010EE66ED7
:102A500087EC1CF0E55289840000000000000000B3
:102A6000899A00000000FC0EDB508A6E0000000016
:102A7000898A0000000093683BD08986898800001D
:102A800000008994010EE66E87EC1CF0E552898403
:102A9000000000008998AA0EE66E550EE66E550EEF
:102AA000E66E2AD8E552E552E552550EE66EAA0EBC
:102AB000E66E2A0EE66E20D8E552E552E552A00EEB
:102AC000E66E550EE66E550EE66E16D8E552E552E8
:102AD000E552936A00000000899A00000000FC0E95
:102AE000DB508A6E00000000898A000000009368B5
:102AF000E552E7CFD9FF1200D9CFE6FFE1CFD9FFEA
:102B0000899889968984000000008994010EE66EF8
:102B100087EC1CF0E552898400000000936AFD0EEA
:102B2000DB508A6E000000008994010EE66E87EC8F
:102B30001CF0E552898400000000FE0EDB508A6E16
:102B4000000000008994010EE66E87EC1CF0E5524F
:102B500089840000000000000000899A0000000045
:102B6000FC0EDB508A6E00000000898A0000000025
:102B700089869368E552E7CFD9FF1200D9CFE6FFE7
:102B8000E1CFD9FFE6520F0EC16E926A9368929A16
:102B9000898A899889868984936AFD0EDB508A6EBA
:102BA000000000008994010EE66E87EC1CF0E552EF
:102BB000898400000000010EE66E87EC1CF0E552EF
:102BC000000000008994010EE66E87EC1CF0E552CF
:102BD000898400000000FE0EDB508A6E010EE66E56
:102BE00087EC1CF0E552000000008994010EE66EAF
:102BF00087EC1CF0E552898400000000010EE66EAF
:102C000087EC1CF0E55200000000898800000000FD
:102C100093688150DF6E000000008998000000007A
:102C2000DF5000D0E552E552E7CFD9FF120079D846
:102C300014DEFF0808E064DE010808E1E66877DEDC
:102C4000E552010813E10001906B1200E6686FDEA7
:102C5000E55200090BE101DE0201406F0001615104
:102C600001E19ED8F00E03D900019B6B12008998F8
:102C7000F1D8800EE66E550EE66EFED8EBD8300E1B
:102C8000F6D80001010E906FFE0EE66E87EC1CF088
:102C9000E55212009ED8E652DDD8900EE66E550E33
:102CA000E66EC6D801E171D8E55298D092D8E652C6
:102CB0009FD8050EE1D8A1D8020EDED8900EE66EA0
:102CC000550EE66E050EB4D801E15FD8E55286D008
:102CD000D9CFE6FFE1CFD9FF898489968998936A95
:102CE000FD0EDB508A6E000000008994010EE66E36
:102CF00087EC1CF0E552898400000000FE0EDB50DA
:102D00008A6E000000008994010EE66E87EC1CF0CC
:102D1000E5528984000000009368E552E7CFD9FFAF
:102D20001200898489968998000000008994010E18
:102D3000E66E87EC1CF0E55289840000000089985B
:102D40008996936A010E8A6E000000008994010E34
:102D5000E66E87EC1CF0E552898400000000200E2E
:102D60008A6E0000000000008994010EE66E87EC78
:102D70001CF0E552898400000000000093681200F6
:102D8000BBDEE552E552E55212006AD8020E666FCC
:102D90000001010E676F0001616F00019B6B120063
:102DA0005FD8010E666F0001676F0001616F12004E
:102DB000E7CFDBFF0001922BDB5000019E259E6FC9
:102DC00000017907DF2A1200D9DEE552E552DF6EF5
:102DD0001200D9CFE6FFE1CFD9FF1200E552E7CFCD
:102DE000D9FF1200EA6A000FE96E020EEA22120011
:102DF000AA0EE66E550EE66E1200550EE66EAA0E8F
:102E0000E66E120000019B6B00019E6BFF0E00013D
:102E1000915D1200FE0EDBCFE6FF3BDDE5520009BF
:102E20001200FE0EDBCFE6FF82DDE5520009120044
:102E300023D8E66A200EE66EC7DFDFCF40F2010E30
:102E4000E66EE66AC1DFDFCF41F2F00E10D8000176
:102E500061511200CDDF10D8D0DF2A0E3CEF17F001
:102E60000001400E626F020E636F00011200E66EF9
:0E2E7000E66AE66AC0EF16F0E66EC0EF16F0F6
:022E7E0004014D
:102E800040511F0B010801E012004051600BE84265
:102E9000E842E842E842E842010801E012004451F9
:102EA00003E0440501E012004151220A31E0030A27
:102EB00024E0010A15E0210A0DE0010A01E01200F8
:102EC0000201710EDC6F000EDD6F080EDF6FE06B2C
:102ED000DE8121D00201710EDC6F000EDD6F1BD090
:102EE00046C4E4F247C4E5F20201D80EE16F040ED5
:102EF000E26FE66BE76BE38F12000201D80EDC6F26
:102F0000040EDD6F070EDF6FE06BC10EDE6F120087
:102F100042C46CF00201DE8F12000401D86BC20EB5
:102F2000D96F010EDA6FDB6BDC6BDD6B080EDE6FC9
:102F30000001616B606B1A0EE66E020EE66EA2EC8B
:102F400011F0E552E5521E0EE66E030EE66EA2EC9F
:102F500011F0E552E55246D900016A6B6B6B120025
:102F60002CD90001606B6851691102E1000E05D097
:102F700034D9EF50800B01E0010E00092DE1FC0E69
:102F8000DBCF0BF02AD9EE52EF50D8800B5405E27C
:102F900024D9EE52FC0EEFCFDBFF606BFC0EDB5052
:102FA000605D19E26051EA6A580FE96E040EEA2288
:102FB000EF50E66E6051E76EFD0EDBCFE9FFFE0ECF
:102FC000DBCFEAFFE750E926000EEA22E552E750A0
:102FD000EF6E602BE3D706D900016051F3D0EDD836
:102FE0000001615107E1E2D8FC0EDBCF66F0010E73
:102FF000676F616FE7D00BD917E1BDD8E7D802E161
:103000000C500BE0010EDBCFE9FFDB2A020EDBCF19
:10301000EAFF01E3DB2AEF50F1E1C8D8DFCF66F029
:103020000001010E676F616F030EE15C02E2E16A6D
:10303000E552E16EC7D0EBD818E19DD8C7D802E1C0
:103040000C500CE0010EDBCFF6FFDB2A020EDBCFCB
:10305000F7FF01E3DB2A0800F550F0E1A7D8DFCF46
:1030600066F00001676B010E616F030EE15C02E226
:10307000E16AE552E16EA6D0A0D8020EE126000179
:103080006A516B1102E1000E08D06AC0E9FF6BC003
:10309000EAFFEF50800B01E0010E00095CE1030E36
:1030A000615D01E1616B615156E0020E615D08E115
:1030B000E66A000EE66EE66AA2D80001030E43D06F
:1030C000610542E1400E0B6E0C6A66510B5C000E0E
:1030D0000C5803E2400EDF6E02D066C0DFFFDF5007
:1030E000665D666F980E646F040E656F010EDFCF2C
:1030F000DBFF67510BE1010EDB5012E062C0F6FF0F
:1031000063C0F7FF0800F55044D8F5D7010EDB5037
:1031100007E062C0E9FF63C0EAFFEF503AD8F6D794
:103120000001665111E16AC0E9FF6BC0EAFFEE528F
:10313000EF500B6E0C6A400E0B1804E10C5002E1CC
:10314000020E01D0030E616FDFCFE6FF980EE66E30
:10315000040EE66E54D8020EE15C02E2E16AE5522A
:10316000E16E30D0030EE66ED6EC11F00B6E050E5C
:10317000E15E0B501200DF6AFD0EDBCF06F0FE0EA3
:10318000DBCF07F0DE5206C0DEFF07C0DDFFDD52F9
:10319000120064C0E9FF65C0EAFFEF6E642B000E09
:1031A0006523622B6323010EDB061200FD0EDBCFCD
:1031B00062F0FE0EDBCF63F01200D9CFE6FFE1CF65
:1031C000D9FF1200E552E7CFD9FF1200DF2ADF5006
:1031D0000B6E0C6AFF0E0B18120068C0E9FF69C085
:1031E000EAFF1200400EE66E580EE66E040EE66E22
:1031F000E66AB8DFF3CF68F0F4CF69F01200010E91
:10320000E66EB0DFF3CF6AF0F4CF6BF01200D5DFDB
:0A321000030EE126000161511200D7
:06321A0000019E6B03C2DF
:10322000F8F202C2F9F204C2FAF20201FB6B010EDB
:10323000FC6F200EFA5D07E3FAC2E6FFF8C2E6FF74
:103240005AD8E552E55225EF19F0D9CFE6FFE1CF84
:10325000D9FF020EE126DF6A010EDB6A0201400E91
:10326000D880FB55000EFC5513E2010EDB6A1AD91B
:1032700025E2200EFA5D03E20DD9EF6801D01AD9DC
:1032800020D90201FB07000EFC5B010EDB2AEFD701
:10329000010EDB6A07D90CE2200E0201FA5D03E29F
:1032A000F9D8EF6801D006D90CD9010EDB2AF2D784
:1032B0000201FB6B010EFC6FFA2BF9070001400EB7
:1032C000626F020E636F0001400E666F0001010E17
:1032D000676F0001616F0201F95103E10001100EF7
:1032E0009B6F020EE15C02E2E16AE552E16EE5529B
:1032F000E7CFD9FF1200D9CFE6FFE1CFD9FFFE0E0D
:10330000DB50070A10E0010A0BE0030A06E0010A9D
:1033100001E00CD0899089920AD08980899207D0E7
:103320008990898204D08980898201D000D08984E3
:10333000898689980A0EE66E87EC1CF0E552936A3E
:103340008A6A000000008994010EE66E87EC1CF08A
:10335000E552898400000000000000008994010EFD
:10336000E66E87EC1CF0E552898400000000FD0E3B
:10337000DB508A6E0A0EE66E87EC1CF0E552000008
:1033800000008994010EE66E87EC1CF0E5528984FA
:103390000000000093688988E552E7CFD9FF12004A
:1033A000D9CFE6FFE1CFD9FFE6528150DF6E0000B2
:1033B00000008994010EE66E87EC1CF0E5528984CA
:1033C00000000000DF5000D0E552E552E7CFD9FF02
:1033D0001200D9CFE6FFE1CFD9FFFE0EDB50070A7E
:1033E00010E0010A0BE0030A06E0010A01E00CD03C
:1033F000899089920AD08980899207D089908982A0
:1034000004D08980898201D000D000000000899416
:10341000010EE66E87EC1CF0E55289840000000086
:10342000E552E7CFD9FF1200D9CFE6FFE1CFD9FFB0
:10343000030EE126FE0EDF6E010EDB683F0EF36E1B
:10344000020EF3CFDBFFD9CFE9FFDACFEAFFEFCFF0
:10345000F6FFEE2AEFCFF7FF000EEE22EFCFF8FFD8
:10346000EE220800F5CF40F2DFCFF6FF010EDBCFF2
:10347000F7FF020EDBCFF8FF0800F5CF41F2F86A44
:10348000030EE15C02E2E16AE552E16EE552E7CF4C
:10349000D9FF1200010EDB50EA6A400FE96E020EFE
:1034A000EA221200400EF36E010EDBCFF4FFF35060
:1034B000F45C120075DFE66EEDDFE552E750EF6E6B
:0E34C0001200E8DFEF5000019E259E6F120003
:0234CE001B5B86
:1034D000324A00303132333435363738394142439D
:1034E000444546000A0A4F3F3F000D0A20507574BC
:1034F00074696E672064657669636520696E746FB0
:1035000020626F6F74206C6F61646572206D6F64F0
:10351000652E200D0A20446973636F6E6E656374B7
:103520002066726F6D2048797065725465726D699E
:103530006E616C2066697273742E200D0A205265CC
:10354000706C75672064657669636520616E6420C0
:103550007573652048494420626F6F746C6F6164B5
:10356000657220746F206C6F6164206669726D777C
:10357000617265200D0A001B5B324A200D0A205043
:1035800072657373205120746F20636F6E66697269
:103590006D20626F6F746C6F61646572206D6F6413
:1035A00065200D0A001B5B324A200D0A205072650F
:1035B0007373205A20746F20636F6E6669726D207A
:1035C000626F6F746C6F61646572206D6F646520EB
:1035D0000D0A000D0A20426F6F746C6F6164657292
:1035E000206D6F64652063616E63656C6C65642E2D
:1035F0002046726F6D2075736572206F722074693A
:083600006D6F7574200D0A00C6
:0836080086D81100D8CFE4FFC1
:10361000E0CFE4FFE46E7FD8E550E5CFE0FFE5CFF3
:10362000D8FF100008D8EFEC0DF028EC08F025D8F2
:103630003CEC18F0F8D70F0EC16E070EB46EF26AAC
:10364000B3EC0DF024EF1BF0949E8B8E816A806AA0
:10365000800E826E899089928B8E948494908B8058
:10366000898A929A92829280928892869284948495
:103670009492949C8B928B9C120004D8200E020191
:10368000C35D12000201FE51FF1104E1100EFE6F36
:10369000270EFF6FFE07000EFF5B6DA204D0FE51E8
:1036A000FF1121E116D00201C3510AE0C30503E076
:1036B000020EC35D02E18B801200040EC35D02E1C5
:1036C0008B901200100EC35D06E10201FE51FF1146
:1036D0000AE18B701200200EC35D05E10201FE516C
:1036E000FF1101E18B701200120012001200120093
:1036F0003FEF17F012008DEF17F06D840201080EF6
:10370000C16F070EC26FC107000EC25BC151C2116B
:10371000FAE16D941200DACFE4FFE652E552E5CF0C
:04372000DAFF1200BA
:0C3724001201000202000008D8040A0094
:1037300001000102000109024300020100C0320938
:10374000040000010202010005240010010424020B
:103750000205240600010524010001070582030873
:10376000000209040100020A0000000705030240EC
:103770000000070583024000000403090434034DE0
:10378000006900630072006F0063006800690070E8
:1037900000200054006500630068006E006F006C3C
:1037A000006F0067007900200049006E0063002E62
:1037B0000038034300440043002000520053002D12
:1037C0000032003300320020004500450043002055
:1037D000004A0033002000500072006F0067007242
:1037E0000061006D0065007200363779377D37B1B2
:0137F00037A1
:0E37F2002A0EF66E100EF76E000EF86E000135
:103800000900F5508B6F0900F5508C6F03E18B6751
:1038100001D03DD00900F550866F0900F550876F43
:103820000900F550886F09000900F550E96E09009C
:10383000F550EA6E090009000900F550896F09008A
:10384000F5508A6F09000900F6CF8DF0F7CF8EF0A2
:10385000F8CF8FF086C0F6FF87C0F7FF88C0F8FF6B
:103860000001895302E18A5307E00900F550EE6E2A
:103870008907F8E28A07F9D78DC0F6FF8EC0F7FFF7
:103880008FC0F8FF00018B07000E8C5BBFD71200C2
:10389000FE0EE3CFE9FFFF0EE3CFEAFFE9CFF3FF30
:1038A000EACFF4FFFB0EE35003E1FC0EE35009E026
:1038B000FB0EE30602E2FC0EE306FD0EE350EE6EA5
:0438C000F1D712002A
:0C38C400FF0EE3500F6EEF0E01D0F30E6C
:1038D000E76EE72E69EF1CF00C0E0E6EE76AE72E1E
:1038E0006FEF1CF00E2E6EEF1CF00F2E67EF1CF02A
:0238F0001200C4
:0E38F20013EE00F023EE00F0F86A0A9CF9ECE9
:0E3900001BF09BEC1CF012EC1BF0FBD712002E
:02390E00FF0EAA
:10391000E350E84E1200000000D000D000D0E82EA6
:04392000FAD71200C0
:0C39240000EE00F00F0EEE6AEA62FDD724
:02393000120083
:043932004F00210021
:0239360012007D
:08393800000000000000000087
:013940000086
:0339410000000083
:0539440000000000007E
:020000040030CA
:0100000024DB
:010001000EF0
:0100020039C4
:010003001EDE
:010005008179
:010006008178
:010008000FE8
:01000900C036
:01000A000FE6
:01000B00E014
:01000C000FE4
:01000D0040B2
:00000001FF
